:100000009AC0CCC025C2B0C0AFC0AEC0ADC0ACC0FD
:10001000ABC0AAC0A9C0A8C0A7C0A6C0A5C0040301
:1000200009045A0368006100660074006D006100F5
:100030006E006E00230073006F006600740077008E
:1000400061007200650020002800770077007700CB
:100050002E00740075002D006300680065006D00BF
:100060006E00690074007A002E00640065002F00A5
:100070007E006800650068006100290022034600D8
:1000800075006E006B005500730062003B004A0073
:100090006F00790073007400690063006B003A031D
:1000A00068006500680061004000680072007A0026
:1000B0002E00740075002D006300680065006D005F
:1000C0006E00690074007A002E00640065003A003A
:1000D0003000300031003000120110010000000833
:1000E000C016DC2700010102030109022200010100
:1000F000008005090400000103000000092101013E
:1001000000012229000705810308000A05010904EE
:10011000A10115002501750195010B010009008160
:1001200002257F75070936810227FFFF0000751041
:1001300009308102C00011241FBECFEDCDBF10E0F9
:10014000A0E6B0E0E4EFF7E002C005900D92A4361F
:10015000B107D9F710E0A4E6B0E001C01D92A13AC2
:10016000B107E1F79AD144C34BCFA82FB92F80E054
:1001700090E041E050EA60956F5F58F42D9138EFC0
:1001800082279795879510F0842795273F5FC8F3BE
:10019000F3CF0895EADF8D939D930895CF93CFB762
:1001A000CF93C395B29BE9F7B29B10C0B29B0EC030
:1001B000B29B0CC0B29B0AC0B29B08C0B29B06C0E7
:1001C000C2B7C2BBC1B3C395C1BBCEC00F92DF9350
:1001D000C0918400DD27C557DF4F012EB29B03C0BD
:1001E000DF910F90E1CF2F930F931F934F932FEF3A
:1001F0004F6F06B302FB20F95F933F9350E03BE063
:1002000065C016B30126502952FDC89556B3012783
:1002100002FB25F92F7306B3B1F05027102712FB0C
:1002200026F906B22230F0F000C016B3012702FB17
:1002300027F90126502906B22430E8F54F772068C7
:1002400016B30000F6CF50274F7D206206B2102F64
:10025000000000C006B300265029102712FB26F923
:1002600006B2E2CF4F7B06B3206400C0DACF01268E
:100270005029167006B269F14E7F2160012F16B326
:1002800028C0002650294D7F06B22260102F29C0B9
:10029000012650294B7F06B22460012F2DC016B3D2
:1002A00001265029477F2860000006B22EC04F7EED
:1002B00006B3206130C0422706B349930026502977
:1002C000102706B24FEF12FB20F9297F16B379F2FF
:1002D000167049F10126502906B2012702FB21F9C7
:1002E000237F06B371F2002650293150D0F006B2B8
:1002F000102712FB22F9277E16B351F2012650294E
:10030000012702FB06B223F92F7C49F2000006B355
:10031000102712FB24F90026502906B22F7939F252
:1003200070CF002717C03B503195C31BD0400881C8
:10033000033CF1F00B34E1F0209182001981110FA0
:100340001213EFCF4A81441F093639F10D3211F0F3
:10035000013E39F7009389003F915F914F911F91C2
:100360000F912F91DF910F90CF91CFBFCF91189523
:1003700000918900002381F310918700112379F502
:1003800034307AF130938700009383001091840019
:100390003BE0311B3093840024C000918700013082
:1003A000F4F40AE54F7049F43091610034FD1AC04D
:1003B00000936100CCE6D0E019C03091620034FDBA
:1003C00011C000936200C7E7D0E010C0052710E01D
:1003D00000C021C0052710E0C89508BB14C03AE54D
:1003E00001C032ED032EC0E0D0E032E017B316605A
:1003F000C29A08B317BB56E020E84FEF20FF05274D
:1004000008BB279517951C3F28F700004552B0F709
:1004100020FF0527279508BB17951C3FB8F62991A3
:100420003A9561F7097F10918800110F08BBC250FF
:10043000D04011F010938200046017B3197F402F51
:10044000497F54E05A95F1F708BB17BB48BB84CFEE
:1004500078941F920F920FB60F9211248F939F934F
:1004600091E090936900B39905C08FEF89BD909397
:10047000660004C080E389BD1092660080916A0026
:1004800090916B0090936800809367009F918F918B
:100490000F900FBE0F901F90189594B714BE479AF7
:1004A00088E181BD11BC11BA93FF0BC086B3867081
:1004B00041F080E48BBF80E385BFC49A789488952F
:1004C000F89480E285BF8BE080BD83EC8ABD80E339
:1004D00089BD82E083BF81E187BB18BA88E085BB14
:1004E00080E68BBF8BB780648BBF8BE480937700F3
:1004F00086B38670E9F388E081BD78948895A895E5
:100500009091870019160CF0C2C020918400809150
:1005100083008D3209F0B1C08AE5809361009B3081
:1005200009F0ABC0ECE0F0E0E21BF109E557FF4F4A
:100530009081892F807609F083C0109275008181A7
:10054000882351F41092760085E790E0909386001E
:100550008093850022E089C0853021F482818093D8
:10056000880082C0863009F050C08381813041F418
:1005700088ED90E0909386008093850022E172C020
:10058000823019F48AEE90E01BC0833051F58281ED
:10059000882341F48EE190E090938600809385005B
:1005A00024E060C0813041F482E290E090938600C4
:1005B000809385002AE556C0823041F48CE790E0B4
:1005C000909386008093850022E24CC0833009F02E
:1005D00048C08EE990E090938600809385002AE3DE
:1005E00041C0813241F48CEF90E09093860080937B
:1005F000850029E037C08232A1F58CE091E090932C
:1006000086008093850029E22DC0883019F48AE89D
:1006100090E00AC0893021F4828180938A0024C04E
:100620008A3041F485E790E09093860080938500BE
:1006300021E01BC08B30C1F48BE48093770014C0A1
:100640009076903289F48181813071F48381813098
:1006500059F486E690E0909386008093850023E02D
:1006600004C020E090EC02C020E090E8878188235D
:1006700039F48681821728F003C080E090E801C039
:10068000822F909365008093600010928700809184
:10069000610084FF49C0809160008F3F09F444C02D
:1006A000182F893008F018E0811B8093600080913A
:1006B000650080FD02C00BE401C003EC8F5F8093F6
:1006C0006500209185003091860086FD05C0D90126
:1006D000912FEDE6F0E011C0ADE6B0E080E090E0F3
:1006E00006C0F901E80FF91FE491ED930196181780
:1006F000C1F705C08D91819391509923D9F7F901E4
:10070000E10FF11DF0938600E09385008DE690E007
:10071000612F40DD183019F08FEF80936000009357
:100720006C001C5F109361009AE086B3867031F410
:100730009150D9F7109288001092820081B38823DB
:1007400051F181B3813079F492B39E50809164006D
:10075000981B993F1CF481B78F5F81BF98301CF0C4
:1007600081B7815081BFF89421B380916A00909144
:100770006B00820F911D90936B0080936A0081B390
:10078000880F90916600890F8093660082B38093F2
:100790006400789411BA8091620084FFAFCE80919A
:1007A0006900882309F4AACE8091620084FF07C003
:1007B0008091770098E889278093770003C08AE5C5
:1007C000809362008091660080937800809167003A
:1007D000809379008091680080937A0088E790E0A8
:1007E00063E0D8DC87E0809362001092690086CED7
:0407F000F894FFCFAB
:0407F400FF5A5A004E
:00000001FF
